:100000000C949C000C94C4000C94C4000C94C40088
:100010000C94C4000C94C4000C94C4000C94C40050
:100020000C94C4000C94C4000C94C4000C94CA0C2E
:100030000C94FE100C94C4000C94C4000C94C400E6
:100040000C94E8130C94C4000C9469160C94C4002E
:100050000C94C4000C94C4000C94C4000C94C40010
:100060000C94C4000C94C400746F6F206D616E79A1
:10007000206F70656E2066696C6573006261642034
:10008000696E707574005941414B00594545454BA7
:100090000053616D706C65207261746520746F6FC0
:1000A0002068696768210000436F6D707265737323
:1000B000696F6E206E6F7420737570706F727465E7
:1000C00064006661696C656420746F2067657420E4
:1000D0006E657720636C7573746572002021212131
:1000E0002000203F3F3F2000000024272A00002559
:1000F000282B000023262904040404040404040219
:1001000002020202020303030303030102040810B4
:100110002040800102040810200102040810200081
:1001200000000700020100000304060000000000B8
:10013000000000004811401211241FBECFEFD4E090
:10014000DEBFCDBF11E0A0E0B1E0EEEAFEE202C00A
:1001500005900D92A232B107D9F714E0A2E2B1E006
:1001600001C01D92A237B107E1F711E0C8E3D1E069
:1001700004C02297FE010E945117C433D107C9F76A
:100180000E9439120C9455170C940000089508959C
:10019000CB010E94EA020895FC01848195810E94AE
:1001A0007C040895EF92FF920F931F93CF93DF93F8
:1001B000EB018A0179010BC0B801C7010E94A616A4
:1001C000009729F4CE010E947C0481E006C0B701AB
:1001D000CE010E948504882379F7DF91CF911F918A
:1001E0000F91FF90EF900895EF92FF920F931F935E
:1001F000DF93CF93CDB7DEB768970FB6F894DEBF25
:100200000FBECDBF8C017E010894E11CF11C97014B
:100210000E94D200882319F420E030E005C0B70125
:10022000C8010E945E089C01C90168960FB6F89447
:10023000DEBF0FBECDBFCF91DF911F910F91FF9019
:10024000EF900895FC01AB016481758182819381F7
:100250000E94F4000895EF92FF920F931F93DF9393
:10026000CF93CDB7DEB768970FB6F894DEBF0FBE59
:10027000CDBF8B017E010894E11CF11CB701FC018C
:10028000848195810E948504882349F04CE050E0E8
:10029000B701C8010E94BD16F801148681E0689676
:1002A0000FB6F894DEBF0FBECDBFCF91DF911F9187
:1002B0000F91FF90EF900895FC01848195810E9439
:1002C00076040895EF92FF920F931F93DF93CF93DD
:1002D000CDB7DEB768970FB6F894DEBF0FBECDBFBF
:1002E0008C017E010894E11CF11CB701FC018281A4
:1002F00093810E942805B701F801828193810E94B1
:100300000F07F8019583848320E0892B09F021E011
:10031000822F68960FB6F894DEBF0FBECDBFCF9187
:10032000DF911F910F91FF90EF9008950F931F930E
:100330008C01FC01808191810E943905F801938331
:10034000828320E0892B09F021E0822F1F910F91F9
:1003500008950F93CF93DF93EC0100E020E030E0AD
:1003600040E050E06BEE7AE081E39AE00E94A5085D
:1003700099838883892B69F40FEF20E030E040E017
:1003800050E06BEE7AE081E39AE00E94A508998341
:10039000888320E088819981892B09F021E0822FD0
:1003A000DF91CF910F9108950E94DB090895FC0120
:1003B000009711F0118210820895DC018C91853E26
:1003C00039F1882329F1F9012081318182819381DA
:1003D0002817390799F444835583668377831B96DE
:1003E0008C911B978F3011F080E205C08C91829523
:1003F000880F807E805E808780E008951B968C91B8
:100400008F3031F02F5F3F4F3183208381E008959B
:1004100081E008950F931F93CF93DF938C01FC012C
:100420008081853E09F48CC0882309F489C0E901E4
:100430008C899D89AE89BF890097A105B10521F4FA
:100440004C8B5D8B6E8B7F8B209709F479C00115E7
:10045000110509F475C0F8018081882309F470C082
:1004600083858F3011F481E06CC0A801D80180E051
:1004700090E0282F3C91303251F0FE01E80FF91F37
:1004800030832F5F019611968830910591F788810E
:10049000853011F485EE8883F80180858032B1F0D3
:1004A000FE01E20FF11D8EE28083822F8F5F2C5FB1
:1004B000FA019085903249F0FE01E80FF11D90831A
:1004C0008F5F4F5F5F4F821799F7282FFE01E20F72
:1004D000F11D1082F80183858D87938D80E0228D38
:1004E00030E0822B932B9F878E87258D30E040E074
:1004F00050E0542F432F322F2227868D90E0A0E02A
:10050000B0E0DC0199278827282B392B4A2B5B2B5D
:10051000848D90E0A0E0B0E0282B392B4A2B5B2B98
:10052000878D90E0A0E0B0E0B82FAA279927882710
:10053000282B392B4A2B5B2B288B398B4A8B5B8BD7
:1005400080E0DF91CF911F910F910895DF93CF93BA
:1005500000D0CDB7DEB7DC010097A1F162307105A4
:1005600088F1ED91FC911197660F771F80E090E084
:1005700016962D913D914D915C911997620F731FC5
:10058000841F951F0190F081E02D22E030E0AE0144
:100590004F5F5F4F09958823A9F09A8180E02981F8
:1005A00030E0282B392B2115310571F08FEF273FD3
:1005B000380741F0C9014096079720F08FEF283F98
:1005C000380710F020E030E0C9010F900F90CF9174
:1005D000DF910895FC01009711F0118210820895B7
:1005E0002F923F924F925F926F927F928F929F9243
:1005F000AF92BF92CF92DF92EF92FF920F931F9331
:10060000DF93CF93CDB7DEB72C970FB6F894DEBF4C
:100610000FBECDBF3C0178876F835A87498700970B
:1006200009F402C1672B09F4FFC0452B09F4FCC093
:10063000DC015A96AD90BD90CD90DC905D975296BE
:100640002D913D914D915C915597E985FA85CF01AA
:10065000A0E0B0E08A0D9B1DAC1DBD1D2817390719
:100660004A075B0740F4B9016A197B097A876987F1
:10067000672B09F4DCC0D301ED91FC91119720891F
:1006800031893A8329835E966D917C915F977C874F
:100690006B87C901A0E0B0E08B839C83AD83BE83F0
:1006A000672BE1F5F3010088F189E02DFC87EB87EA
:1006B000EF2B39F4A114B104C104D10409F4B7C07B
:1006C000B3C0A114B104C104D10441F18601750184
:1006D0002B803C804D805E805094409430942094D8
:1006E000211C311C411C511C10C06B857C85D30121
:1006F0008D919C910E94A6029C878B87892B09F47F
:1007000093C0E20CF31C041D151D6B817C818D814F
:100710009E81E616F7060807190738F7C601B501E6
:100720002B813C814D815E810E9412172B018984AF
:100730009A84D301ED91FC91A980BA80A418B508E0
:100740008A149B0408F45401C080D180720100E037
:1007500010E086899789A08DB18DE80EF91E0A1FD9
:100760001B1FEB85FC853297BF0180E090E032963D
:10077000FC87EB872B813C814D815E810E94CC16EA
:10078000E60EF71E081F191FD601ED91FC91950189
:100790004F815885C801B7010995882361F18A18EE
:1007A0009B08C501A0E0B0E0F301228D338D448D9C
:1007B000558D280F391F4A1F5B1FD3015A962D9361
:1007C0003D934D935C935D97C501840D951DE98123
:1007D000FA818E179F07B0F06B857C858D919C9177
:1007E0000E94A6029C878B87892B51F4D3015F96C8
:1007F0001C921E925E9749855A854819590919C05D
:10080000442455242B853C85F301378F268F811492
:10081000910439F06F8178856A0D7B1D78876F832D
:1008200088CF49855A8505C04FEF5FEF02C040E091
:1008300050E0CA012C960FB6F894DEBF0FBECDBFB4
:10084000CF91DF911F910F91FF90EF90DF90CF90AC
:10085000BF90AF909F908F907F906F905F904F90E0
:100860003F902F900895CF93DF93FC01EB01009709
:10087000C9F161157105B1F1828D938DA48DB58D8E
:10088000413051F0413018F0423061F50AC0288102
:1008900039814A815B8111C0288139814A815B811C
:1008A00008C0288139814A815B8182899389A48922
:1008B000B589280F391F4A1F5B1F82899389A48934
:1008C000B58982179307A407B50760F0228F338F8D
:1008D000448F558F178E168E288339834A835B8306
:1008E00081E001C080E0DF91CF910895FC01009785
:1008F00011F0118210820895FC01009711F480E03C
:100900000895138E128E81E008952F923F924F9298
:100910005F926F927F928F929F92AF92BF92CF928F
:10092000DF92EF92FF920F931F93DF93CF93CDB798
:10093000DEB7A9970FB6F894DEBF0FBECDBF3C015E
:100940002B01009709F44AC06115710509F446C0EE
:10095000FC0180899189892B09F040C0228D338D5B
:10096000A081B1811097B9F1ED91FC91119722808E
:100970003380AE014F5F5F4F89E0FA0111928A9593
:10098000E9F73C832B8352966D917D918D919C91DB
:10099000559756960D911C915797061B170B6A0198
:1009A0002DEDE22E21E0F22E20E230E0AE01465F96
:1009B0005F4FF1010995882371F08D809E80AF8093
:1009C000B88481149104A104B10429F021C0F2017A
:1009D00080818823A9F5F301138E128E80E0A996F9
:1009E0000FB6F894DEBF0FBECDBFCF91DF911F9140
:1009F0000F91FF90EF90DF90CF90BF90AF909F90BE
:100A00008F907F906F905F904F903F902F900895C0
:100A100088E1F20111928A95E9F7098562019AE06D
:100A2000E92E92E0F92E10E020E230E0AE01465FC0
:100A30005F4FC501B401F1010995882361F2C7CF69
:100A4000F301828D938D0196938F828F81E0C7CFC2
:100A5000FB01892B61F06115710549F088E1DB012B
:100A60001D928A95E9F780E1858781E0089580E00D
:100A700008952F923F924F925F926F927F928F9242
:100A80009F92AF92BF92CF92DF92EF92FF920F931D
:100A90001F93DF93CF93CDB7DEB7E0970FB6F894EF
:100AA000DEBF0FBECDBF6C01009709F490C1ABC192
:100AB000EAE7F1E08AE1DF011D928A95E9F7D09239
:100AC0007B01C0927A01D60119962D913D914D91ED
:100AD0005C911C9719E0220F331F441F551F1A9574
:100AE000D1F72AA33BA34CA35DA3CA01B901655F5B
:100AF0007F4F8F4F9F4FED91FC9129E130E0AE0188
:100B00004F5F5F4F0995882309F484C1A9804A800B
:100B1000BB81BEA30C81FD801E813F815884698406
:100B20007A849D8580E02C85E22FF0E0E82BF92B7C
:100B30008E883F88288DE98C309709F46BC1432D4E
:100B400050E060E070E0962F852F742F662769A72C
:100B50007AA78BA79CA7822F90E0A0E0B0E0BC0111
:100B60005527442789A59AA5ABA5BCA5842B952B11
:100B7000A62BB72B482D50E060E070E0842B952B1E
:100B8000A62BB72B89A79AA7ABA7BCA78E2D90E061
:100B9000A0E0B0E0782F66275527442789A59AA5BD
:100BA000ABA5BCA5842B952BA62BB72B89A79AA701
:100BB000ABA7BCA70097A105B10589F4972D80E0EC
:100BC000662D70E0682B792B6115710509F422C13F
:100BD000CB01A0E0B0E089A79AA7ABA7BCA7942D52
:100BE00080E02A2C3324282A392A952D80E0A32F4F
:100BF000B0E0A82BB92BB8A7AFA39F2D80E0202F82
:100C000030E0822B932B9C0140E050E02A8F3B8FF9
:100C10004C8F5D8FBF0180E090E0212F30E040E0FD
:100C200050E00E94CC166E8F7F8F88A399A3E9A411
:100C3000FAA40BA51CA54A8D5B8D6C8D7D8DE41AE5
:100C4000F50A060B170B6E8D7F8D88A199A1E61A08
:100C5000F70A080B190BC10101972FA138A5B5E0C0
:100C6000220F331FBA95E1F7820F931FB1010E9443
:100C7000EB1680E090E0E61AF70A080B190B7EA14C
:100C8000272F30E040E050E0C801B7010E94121762
:100C900029013A01D301C201855F9F40A040B040C5
:100CA0008050904FA040B04008F0B4C086E0D6011C
:100CB00018968C93ACE78A2EA1E09A2E88E1F40175
:100CC00011928A95E9F75101CC24DD2469A57AA512
:100CD0008BA59CA5A60195010E94CC1660937C0172
:100CE00070937D0180937E0190937F01C601B501D1
:100CF0002A8D3B8D4C8D5D8D0E94CC167B018C0125
:100D00002AA13BA14CA15DA1E20EF31E041F151FF9
:100D1000E0928001F092810100938201109383019F
:100D200042E050E060E070E0440E551E661E771E03
:100D3000440C551C661C771C40928401509285011E
:100D40006092860170928701309289012092880119
:100D50005EA1852F90E0BC01269EC001279E900DCC
:100D6000369E900D112490938B0180938A016E8D95
:100D70007F8D88A199A1A60195010E94CC166E0DC8
:100D80007F1D801F911F60938C0170938D01809354
:100D90008E0190938F01AFA1B8A59D0140E050E076
:100DA000E5E0220F331F441F551FEA95D1F7620F6C
:100DB000731F841F951F609390017093910180931E
:100DC00092019093930194012250304002C020E0A0
:100DD00030E0C901E0960FB6F894DEBF0FBECDBF7C
:100DE000CF91DF911F910F91FF90EF90DF90CF9007
:100DF000BF90AF909F908F907F906F905F904F903B
:100E00003F902F90089580917A0190917B01892BDA
:100E1000F1F64ECE10927B0110927A01D8CFCF938B
:100E2000DF939C01DB01009729F16115710511F138
:100E30001D968C911D9784FF1DC080912201909179
:100E40002301892B19F4E2E2F1E008C080913E0110
:100E500090913F01892B71F4EEE3F1E0EF012296CE
:100E600088E10D9009928150E1F731832083138E40
:100E7000128E02C0E0E0F0E0CF01DF91CF91089543
:100E80002F923F924F925F926F927F928F929F929A
:100E9000AF92BF92CF92DF92EF92FF920F931F9388
:100EA000DF93CF93CDB7DEB72A970FB6F894DEBFA6
:100EB0000FBECDBF4C017C836B831A01009709F4F0
:100EC000DEC0672B09F4DBC04115510509F4D7C01A
:100ED000DC015A96ED90FD900D911C915D9780E09C
:100EE0009EEFAFEFBFEFE822F9220A231B23D401C4
:100EF0005A96ED92FD920D931C935D9752962D910B
:100F00003D914D915C9155972E153F054007510736
:100F100008F4B8C0C101A0E0B0E08E0D9F1DA01F75
:100F2000B11F281739074A075B0728F419012E1843
:100F30003F0809F4A7C0D401ED91FC9111972089D5
:100F400031893A8329835E968D919C915F979A8728
:100F50008987290166247724892BD9F550960D902D
:100F6000BC91A02DBA87A987AB2B39F4E114F10409
:100F70000105110509F486C082C0E114F1040105E0
:100F8000110539F15701680188279927DC01841977
:100F90009509A609B7098D839E83AF83B88714C0CE
:100FA00069857A85D4018D919C910E94A6029A87C9
:100FB0008987892B09F463C08D819E81AF81B885B3
:100FC000A80EB91ECA1EDB1EA414B504C604D7049D
:100FD00038F7510191E0291692E0390618F0A12C5A
:100FE00082E0B82EC801B701A30192010E94121736
:100FF0007B0129813A81261B370B65012A153B05A8
:1010000008F4690100E010E0D401ED91FC918689BB
:101010009789A08DB18DE80EF91E0A1F1B1FE98567
:10102000FA853297BF0180E090E03296FA87E9872F
:10103000A30192010E94CC16E60EF71E081F191F8D
:1010400096014B815C81C801B7010E943D0C892B40
:10105000C9F0960140E050E0F401828D938DA48D9B
:10106000B58D820F931FA41FB51F828F938FA48FFE
:10107000B58F29853A85378F268FA50105C04FEF9B
:101080005FEF02C040E050E0CA012A960FB6F89424
:10109000DEBF0FBECDBFCF91DF911F910F91FF90AB
:1010A000EF90DF90CF90BF90AF909F908F907F9008
:1010B0006F905F904F903F902F900895CF93DF9364
:1010C0009C01FB01009731F06115710519F08585D0
:1010D00084FF2CC060E08CE790E003C060E088E60D
:1010E00090E00E94A60C20E030E0C901DF91CF9192
:1010F0000895CCE5D1E0DF0188E10D90099281509F
:10110000E1F730935B0120935A0110927401109221
:1011100075011092760110927701868597859093DC
:101120007901809378012AE531E0DFCF80915A017F
:1011300090915B01892B91F6DCCFFC01009711F4B3
:1011400080E00895108681E008958F929F92AF927B
:10115000BF92CF92DF92EF92FF920F93DF93CF93E4
:10116000CDB7DEB760970FB6F894DEBF0FBECDBF28
:101170007C016B015A014901009709F493C0611584
:10118000710509F48FC004300CF08CC007FD1DC040
:10119000602F772767FD7095E4E0660F771FEA956B
:1011A000E1F762547E4F882777FD8095982F20E1E4
:1011B00030E0AE014F5F5F4FF7010995882309F4D6
:1011C00071C08D81882309F46DC080919C018823B2
:1011D00009F068C07CC08D8180939C012A8530E035
:1011E00040E050E0542F432F322F22278B8590E090
:1011F000A0E0B0E0DC0199278827282B392B4A2B67
:101200005B2B898590E0A0E0B0E0282B392B4A2B9E
:101210005B2B8C8590E0A0E0B0E0B82FAA2799273F
:101220008827282B392B4A2B5B2B20939D01309349
:101230009E0140939F015093A0012E8530E040E035
:1012400050E0542F432F322F22278F8590E0A0E0CB
:10125000B0E0DC0199278827282B392B4A2B5B2B00
:101260008D8590E0A0E0B0E0282B392B4A2B5B2B3A
:10127000888990E0A0E0B0E0B82FAA2799278827B6
:10128000282B392B4A2B5B2B2093A1013093A201F1
:101290004093A3015093A40103C08FEF80939C015E
:1012A0009F0102C020E030E0C90160960FB6F894BB
:1012B000DEBF0FBECDBFCF91DF910F91FF90EF90BA
:1012C000DF90CF90BF90AF909F908F900895E4E90A
:1012D000F1E081E1DF011D928A95E9F7F092950135
:1012E000E0929401D0929701C0929601B092990138
:1012F000A092980190929B0180929A0107FF6BCF78
:10130000CCCF81E0089581E00895282F8FEF8EBD26
:101310000DB407FEFDCF8DB58F778DBD8EB5822FB5
:1013200080648EBD0DB407FEFDCF8DB58F778DBD6A
:10133000872F9927AA27BB278EBD0DB407FEFDCFA7
:101340008DB58F778DBDCB01AA27BB278EBD0DB480
:1013500007FEFDCF8DB58F778DBDBB27A72F962FAD
:10136000852F8EBD0DB407FEFDCF8DB58F778DBD5A
:101370004EBD0DB407FEFDCF8DB58F778DBD2223F9
:1013800011F08FEF01C085E98EBD0DB407FEFDCFD2
:101390008DB58F778DBD90E02FEF2EBD0DB407FE7C
:1013A000FDCF8DB58F778DBD8EB58F3F19F49F5FC3
:1013B0009A3099F70895CF93DF93239A259A229A2A
:1013C00024982A9A83E58CBD8DB58E7F8DBD20E053
:1013D00030E09FEF9EBD0DB407FEFDCF8DB58F773A
:1013E0008DBD8EB52F5F3F4F2A30310599F72A9872
:1013F000C0E0D0E040E050E060E070E080E00E94BB
:101400008509813031F081E0CF3FD807E1F02196A6
:10141000F1CFC0E0D0E040E050E060E070E081E07B
:101420000E94850980FF06C08FE7CF3FD80759F09B
:101430002196F1CF40E052E060E070E080E10E9450
:101440008509882319F02A9A80E008C02A9A8CB569
:101450008C7F8CBD8DB581608DBD81E0DF91CF919A
:1014600008958F929F92AF92BF92DF92EF92FF9278
:101470000F931F93CF93DF937B018C015A01E901F6
:10148000DD24DA94812C42E0942E5EC02A98B801C3
:10149000A70140705E7F81E10E948509882319F0D1
:1014A0002A9A80E055C0DEBC0DB407FEFDCF8DB595
:1014B0008F778DBD8EB58E3FB1F7A7015170B40106
:1014C000641B750BC617D70708F4BE01FB01E40FB8
:1014D000F51F20E030E0DEBC0DB407FEFDCF8DB57A
:1014E0008F778DBD8EB52417350730F02E173F0747
:1014F00018F4D5018D935D012F5F3F4FB2E020308E
:101500003B0749F7DEBC0DB407FEFDCF8DB58F77E5
:101510008DBD8EB5DEBC0DB407FEFDCF8DB58F77CA
:101520008DBD8EB52A9ADEBC0DB407FEFDCF8DB5FC
:101530008F778DBD8EB5C61BD70BCB01A0E0B0E079
:10154000E80EF91E0A1F1B1F209709F09FCF81E0AC
:10155000DF91CF911F910F91FF90EF90DF90BF909F
:10156000AF909F908F9008952091000130910101DC
:101570009FEF0AC09EBD0DB407FEFDCF8DB58F77DE
:101580008DBD8EB52F5F3F4F82E02030380790F33E
:101590008FEF8EBD0DB407FEFDCF8DB58F778DBD5E
:1015A0008EB58FEF8EBD0DB407FEFDCF8DB58F7755
:1015B0008DBD8EB52A9A8FEF8EBD0DB407FEFDCF7F
:1015C0008DB58F778DBD8EB58FEF9FEF9093010115
:1015D0008093000108952F923F924F925F926F92F5
:1015E0007F928F929F92AF92BF92CF92DF92EF92B3
:1015F000FF920F931F93DF93CF93CDB7DEB72C9756
:101600000FB6F894DEBF0FBECDBF4B015C011A01CF
:101610003C872B872801FE82ED82D886CF82411538
:10162000510509F4DAC02115310509F4D6C00217B5
:10163000130708F4D2C0EF2809F4CFC02A983095D8
:1016400021953F4F3A87298784011170D501C40144
:1016500080709E7F89839A83AB83BC83AC01BD017C
:1016600081E10E948509882311F02A9AB6C09FEF74
:101670009EBD0DB407FEFDCF8DB58F778DBD8EB5A8
:101680008E3FA9F720E030E00BC0AFEFAEBD0DB448
:1016900007FEFDCF8DB58F778DBD8EB52F5F3F4F88
:1016A0002017310790F3E12C52E0F52EE01AF10AF1
:1016B0003701EB85FC856E1A7F0A6201CE1ADF0ABC
:1016C00000E012E00E191F092B853C85E216F30697
:1016D00048F14216530630F1F10120E030E00CC031
:1016E0008FEF8EBD0DB407FEFDCF8DB58F778DBD0D
:1016F0008EB581932F5F3F4FAB85BC852A173B0783
:1017000078F3A80160E070E0480D591D6A1D7B1D4B
:101710002F813885C101ED81FE810995882321F44F
:1017200091E026C090E024C02B853C85E21AF30AA4
:10173000421A530A61147104A9F389859A85680EC7
:10174000791EC80ED91E020F131FC9018C0D9D1DD5
:10175000892B09F0B9CFE6CFAFEFAEBD0DB407FED0
:10176000FDCF8DB58F778DBD8EB50894E108F1085A
:10177000E114F10489F7BFEFBEBD0DB407FEFDCF44
:101780008DB58F778DBD8EB5EFEFEEBD0DB407FE35
:10179000FDCF8DB58F778DBD8EB52B853C854216DF
:1017A000530678F0992369F489809A80AB80BC80D5
:1017B00080E092E0A0E0B0E0880E991EAA1EBB1E59
:1017C00043CF2A9A8FEF8EBD0DB407FEFDCF8DB5A6
:1017D0008F778DBD8EB581E001C080E02C960FB66D
:1017E000F894DEBF0FBECDBFCF91DF911F910F9157
:1017F000FF90EF90DF90CF90BF90AF909F908F9031
:101800007F906F905F904F903F902F900895FC01D4
:1018100020910001309101014FEF2F3F340731F447
:1018200060E086E890E00E94A60CFFCFCB01820F1B
:10183000931F8150924020F060E072E0621B730BB6
:1018400020E030E04FEF14C04EBD0DB407FEFDCFD9
:101850008DB58F778DBD8EB581938091000190916C
:101860000101019690930101809300012F5F3F4F8A
:101870002617370748F3CB010895CF92DF92EF92F6
:10188000FF920F931F93CF93DF937B018C016A012B
:1018900080910001909101018F5F9F4F31F060E0D6
:1018A0008BE890E00E94A60CFFCFE90182E0213096
:1018B000380710F0C0E0D2E02A9880E09EEFAFEF4A
:1018C000BFEFE822F9220A231B23B801A70181E117
:1018D0000E948509882321F02A9AC0E0D0E02CC01C
:1018E0009FEF9EBD0DB407FEFDCF8DB58F778DBDEB
:1018F0008EB58E3FB1F710920101109200012FEFCB
:1019000014C02EBD0DB407FEFDCF8DB58F778DBDF4
:101910008EB5D6018D936D018091000190910101EA
:1019200001969093010180930001809100019091B4
:1019300001018C179D0728F3CE01DF91CF911F91F4
:101940000F91FF90EF90DF90CF9008950F931F932A
:10195000CF93DF93EC01062F10E005C084EE93E0F7
:101960000E9459121F5FFE01E10FF11D6491662371
:10197000A9F7002351F06AE084EE93E00E9461121F
:101980006DE084EE93E00E946112DF91CF911F9190
:101990000F9108951F920F920FB60F9211242F935B
:1019A0003F934F938F939F93AF93BF93EF93FF9387
:1019B000E091A501F091A601309709F4A8C020910B
:1019C000AB033091AC038091AD039091AE03281727
:1019D000390709F047C08091B0038823B9F180919D
:1019E000A7039091A80327EA32E041E0873A9407E1
:1019F00049F43093A8032093A7039093AA038093FC
:101A0000A9030AC087EA91E09093A8038093A703F3
:101A10003093AA032093A9038091A7039091A80370
:101A20009093AC038093AB0380509F4F9093AE0391
:101A30008093AD031092B0038091AF03882391F49B
:101A400080916F00846080936F000CC081899289BF
:101A5000A389B4890196A11DB11D818B928BA38BA3
:101A6000B48B55C05A985C985B9A5B985C9A5B9A69
:101A70005B985B9A5B985B9A5B988781803119F5DC
:101A8000E091AB03F091AC038181805890E087FF37
:101A900002C05C9A01C05C985B9A5B989F5F98302B
:101AA00011F0880FF4CF908180E097FF02C05C9A1C
:101AB00001C05C985B9A5B988F5F843011F0990F3E
:101AC000F4CF32961DC08830F9F4E091AB03F09169
:101AD000AC03908180E097FF02C05C9A01C05C98E3
:101AE0005B9A5B988F5F883011F0990FF4CF5B9A07
:101AF0005B985B9A5B985B9A5B985B9A5B98319674
:101B0000F093AC03E093AB035A9A5D985D9AFF9112
:101B1000EF91BF91AF919F918F914F913F912F91F5
:101B20000F900FBE0F901F90189508950895DC0137
:101B30005696ED91FC9157976289738984899589AE
:101B400008959A01AB0160E074E284EF90E00E9496
:101B5000121730938900209388000895CF93DF9364
:101B6000EC0180916F008D7F80936F008D898823B9
:101B700019F00E94B40A1D8AE091A501F091A60116
:101B8000108A1092A6011092A501DF91CF910895BD
:101B90000F931F93DF93CF9300D000D0CDB7DEB764
:101BA0008C01407049835A836B837C83DC0150969F
:101BB0008C91882351F0F894F8018589882329F0C5
:101BC0000E94B40AD80155961C9240E0BE016F5F96
:101BD0007F4FF801868997890E943304D801569671
:101BE000ED91FC91579782899389A489B5892981C0
:101BF0003A814B815C81821B930BA40BB50BF801DE
:101C000080879187A287B38778940F900F900F9069
:101C10000F90CF91DF911F910F910895CF92DF9296
:101C2000EF92FF920F931F93DF93CF93CDB7DEB761
:101C300028970FB6F894DEBF0FBECDBF8C016B01A5
:101C400044E050E07E010894E11CF11CB701C6019C
:101C50000E94F002049709F0F0C044E050E062E016
:101C600071E0C7010E94AF16009709F0E6C0F5C009
:101C700044E050E067E071E0CE0105960E94AF16A7
:101C8000009709F0DAC0F2C044E050E06CE071E087
:101C9000C7010E94AF16009709F0CFC0F0C0542FC3
:101CA000432F322F22278081280F311D411D511DC6
:101CB0003197EC17FD0799F7F80124873587468798
:101CC0005787203131054105510509F0B6C048E07C
:101CD00050E0BE016F5F7F4FC6010E94F00208977F
:101CE00009F0ABC08A8190E0A0E0B0E0BA2FA92F44
:101CF000982F88272981820F911DA11DB11D019761
:101D0000A105B10521F061E088EA90E084C08C81F2
:101D100090E0A0E0B0E02227382F492F5A2F8B8186
:101D2000280F311D411D511D23303105410551053D
:101D300008F083C0F8012083FE013896BE016C5F75
:101D40007F4F542F432F322F22278081280F311DA0
:101D5000411D511D3197E617F70799F7F8012183C7
:101D600032834383548348E050E0BE016F5F7F4F6E
:101D7000C6010E94F002089709F05FC08E8190E0D2
:101D8000A0E0B0E0BA2FA92F982F88272D81820FCD
:101D9000911DA11DB11DF80196838583888590E072
:101DA000A0E0B0E02227382F492F5A2F8F81280F2B
:101DB000311D411D511D213131054105510508F0ED
:101DC0003CC0278381819281A381B4818332F6E56F
:101DD0009F07F0E0AF07F0E0BF0718F0293040F0B0
:101DE0000CC081589E43A040B04050F0293040F0D4
:101DF000FF24F8018081823020F0FF24F39401C099
:101E0000FF2461E087EA90E00E94A60CFF2031F0F9
:101E100061E081E990E00E94A60C0FC0F8011086F5
:101E2000118612861386D78AC68A118A128A138A65
:101E3000148A108A158A81E001C080E028960FB6C6
:101E4000F894DEBF0FBECDBFCF91DF911F910F91F0
:101E5000FF90EF90DF90CF90089548E050E0B701F9
:101E6000C6010E94F002089741F702CF44E050E01B
:101E7000B701C6010E94F0020497F9F605CFF801F8
:101E8000148615861686178644E050E0B701C60111
:101E90000E94F002049789F6F8012485358546856D
:101EA0005785FE013496FBCEAF92BF92CF92DF9260
:101EB000EF92FF920F931F93DF93CF9300D000D048
:101EC0000F92CDB7DEB76C015B01F42EE52EFC015D
:101ED00080859185A285B3850097A105B105D1F5CF
:101EE00044E050E08E010F5F1F4FB801868997894B
:101EF0000E94F002049709F0F5C01D8244E050E012
:101F0000B801D60156968D919C9157970E94F00288
:101F1000049709F0E7C0F601108611861286138631
:101F2000FE01349620E030E040E050E0542F432F93
:101F3000322F22278081280F311D411D511D3197DD
:101F4000EC17FD0799F7D60118962D933D934D9305
:101F50005C931B978F2D9E2D9C017901B2E021305F
:101F60003B0718F0E12C72E0F72EF6012085318551
:101F700042855385C701A0E0B0E0281739074A071A
:101F80005B0708F47901D6015696ED91FC915797BD
:101F9000828D938DA48DB58D9170A070B0700097D7
:101FA000A105B105D1F4D60155968C918823A9F4E9
:101FB000A701B501CF010E9440078C018E159F0536
:101FC00041F060E082EE90E00E94A60C0E94B40A0C
:101FD0008BC081E0F601858B73C0D60155968C913C
:101FE000882309F463C0B701C5010E94070C5C0196
:101FF0008E159F0539F060E08CED90E00E94A60CF4
:102000000E94B40AD6015696ED91FC915797C501EE
:10201000A0E0B0E0228D338D448D558D820F931F4B
:10202000A41FB51F828F938FA48FB58F9170A0705E
:10203000B0700097A105B10509F041C00E94B40A33
:10204000F601158A06891789D801ED90FC90119741
:10205000F7012089318940E050E05A966D917D91D9
:102060008D919C915D970E941217611571058105F4
:10207000910529F5D8015E966D917C915F97C70116
:102080000E94A602F801978F868F892BC1F4D60192
:102090005696ED91FC915797178E168E61E082EC63
:1020A00090E00E94A60C0FEF1FEF1EC0A701B50124
:1020B000CF010E94F0028E159F05A1F401C07501A9
:1020C000970140E050E0F60180859185A285B385B7
:1020D000821B930BA40BB50B80879187A287B387D4
:1020E000870102C000E010E0C8010F900F900F9030
:1020F0000F900F90CF91DF911F910F91FF90EF9074
:10210000DF90CF90BF90AF900895CF92DF92EF9283
:10211000FF920F931F93CF93DF93EC01C980DA8076
:10212000EB80FC809093A6018093A50107EA11E063
:102130001093AC030093AB0342E050E0B8010E945F
:10214000540F892B09F451C08091AB039091AC03DB
:1021500002969093AE038093AD03EE89FF89828D42
:1021600040E051E0481B5109B8016E5F7F4F8091FC
:10217000A5019091A6010E94540F9C010097A9F11E
:102180008091AD039091AE03820F931F9093AE03A5
:102190008093AD0340E051E067EA72E08091A501D1
:1021A0009091A6010E94540F81E08093B003888B28
:1021B0001092800089E08093810060E074E284EFF7
:1021C00090E0A70196010E94121730938900209396
:1021D000880081E090E090938B0080938A0080914A
:1021E0006F00826080936F007894DF91CF911F9190
:1021F0000F91FF90EF90DF90CF9008951F920F9274
:102200000FB60F9211242F933F934F935F936F93C9
:102210007F938F939F93AF93BF93EF93FF9380919F
:102220006F008B7F80936F008091B0038823F9F457
:1022300081E08093AF0378946091A9037091AA0321
:1022400040E051E08091A5019091A6010E94540FB9
:10225000892B31F48091A5019091A6010E94AE0DC9
:10226000F8941092AF0381E08093B0037894FF91CB
:10227000EF91BF91AF919F918F917F916F915F91FE
:102280004F913F912F910F900FBE0F901F90189577
:1022900083EB93E00E94C7008BEB93E00E94960DC6
:1022A00008950F931F93BC0183EB93E00E942201DA
:1022B0009093BA038093B9030BEB13E0BC01C80100
:1022C0000E940E0EC8010E9485101F910F91089563
:1022D0000F931F9381E191E00E94511110E000E003
:1022E00048C0112339F468EE73E080E090E00E946A
:1022F000531402C0153128F460E371E080E090E0EF
:102300001FC0812F85518E3128F468E670E080E08F
:1023100090E016C0812F8353823828F468E170E082
:1023200080E090E00DC0812F855B823328F460E16E
:1023300070E080E090E004C068E070E080E090E051
:102340000E9453141F3F21F0002331F41F5F09C086
:10235000002331F401E005C0112311F400E001C0B5
:102360001150612F66956695669570E086E00E9433
:10237000E6148091CB03882309F0B3CF6091B903B1
:102380007091BA0383EB93E00E94C80060E070E0B4
:1023900086E00E94E6141F910F9108950F931F93FA
:1023A000DF93CF93CDB7DEB72D970FB6F894DEBF8E
:1023B0000FBECDBF83EB93E00E94CC008E010F5F78
:1023C0001F4FB80183EB93E00E942B01882379F41F
:1023D00083EB93E00E94CC002D960FB6F894DEBFFD
:1023E0000FBECDBFCF91DF911F910F910895B8011E
:1023F00084EE93E00E94A812E4CF40E855E260E04A
:1024000070E084EE93E00E94541261E082E00E944A
:102410003A1561E083E00E943A1561E084E00E9491
:102420003A1561E085E00E943A1561E086E00E947D
:102430003A1583EB93E00E94D4018823C9F083EB23
:1024400093E00E94A901882399F083EB93E00E9416
:102450009601882369F083EB93E00E946201882350
:1024600039F00E94CE1160E070E086E00E94E61430
:1024700008950E948B140E94FD110E946811FDCFE7
:102480008FE191E09093E5038093E4030895862F14
:102490000E94281608950E94601608950E94411611
:1024A00008950E9430160895CB01BA010E94EF15DD
:1024B0000895DC01ED91FC910190F081E02D0995EA
:1024C0000895DC01ED91FC910190F081E02D0995DA
:1024D00008950F931F93CF93DF938C01EB0109C0F5
:1024E0002196D801ED91FC910190F081E02DC80179
:1024F000099568816623A1F7DF91CF911F910F9114
:1025000008950F931F938C01DC01ED91FC910190D4
:10251000F081E02D6DE00995D801ED91FC910190DD
:10252000F081E02D6AE0C80109951F910F9108958F
:102530000F931F938C01DC01ED91FC910190F081D0
:10254000E02D0995C8010E9481121F910F910895F5
:102550000F931F938C010E946912C8010E9481127F
:102560001F910F9108950F931F938C01DC01ED9142
:10257000FC910190F081E02D0995C8010E94811223
:102580001F910F9108952F923F924F925F926F92F9
:102590007F928F929F92AF92BF92CF92DF92EF92F3
:1025A000FF920F931F93DF93CF93CDB7DEB7A09722
:1025B0000FB6F894DEBF0FBECDBF1C016A017B01D0
:1025C000411551056105710549F4DC01ED91FC915E
:1025D0000190F081E02D60E3099554C0882499248E
:1025E0005401422E55246624772401E010E00C0F9C
:1025F0001D1F080D191DC701B601A30192010E94FC
:102600001217F80160830894811C911CA11CB11C55
:10261000C701B601A30192010E941217C901DA0194
:102620006C017D01C114D104E104F104F1F681E0F3
:10263000E82EF12CEC0EFD1EE80CF91C3E0108946E
:10264000611C711CD501C4010197A109B1096C017C
:10265000C818D90814C0F601EE0DFF1D60816A305C
:1026600010F4605D01C0695CD101ED91FC910190B5
:10267000F081E02DC10109950894E108F1086E147C
:102680007F0449F7A0960FB6F894DEBF0FBECDBF0A
:10269000CF91DF911F910F91FF90EF90DF90CF903E
:1026A000BF90AF909F908F907F906F905F904F9072
:1026B0003F902F9008952AE00E94C31208950F932F
:1026C0001F938C010E945B13C8010E9481121F910D
:1026D0000F910895AB0160E070E00E945B130895D4
:1026E0000F931F938C01AB0160E070E00E945B13BD
:1026F000C8010E9481121F910F910895EF92FF92DD
:102700000F931F93CF93DF93EC017A018B0177FF37
:102710000FC0E881F9810190F081E02D6DE209950B
:1027200010950095F094E094E11CF11C011D111D21
:102730002AE0B801A701CE010E94C312DF91CF9118
:102740001F910F91FF90EF9008950F931F938C01AD
:102750000E947E13C8010E9481121F910F9108955B
:10276000AB01662757FD6095762F0E947E13089572
:102770000F931F938C01AB01662757FD6095762F51
:102780000E947E13C8010E9481121F910F9108952B
:10279000DC012115310541F4ED91FC910190F081AE
:1027A000E02D642F099508952A30310519F40E940F
:1027B0007E1308950E94C31208950F931F938C01F6
:1027C0000E94C813C8010E9481121F910F910895A1
:1027D0001F920F920FB60F9211242F938F939F93F6
:1027E000AF93BF938091E6039091E703A091E80334
:1027F000B091E9038050904CAF4FBF4F8093E603F8
:102800009093E703A093E803B093E90327C0809176
:10281000E6039091E703A091E803B091E9038058A3
:102820009E43A040B0408093E6039093E703A093BB
:10283000E803B093E9038091EA039091EB03A09140
:10284000EC03B091ED030196A11DB11D8093EA0345
:102850009093EB03A093EC03B093ED038091E60318
:102860009091E703A091E803B091E90381589E435A
:10287000A040B04060F6BF91AF919F918F912F9192
:102880000F900FBE0F901F9018958FB7F89420915E
:10289000EA033091EB034091EC035091ED038FBFBD
:1028A000B901CA010895EF92FF920F931F937B0124
:1028B0008C018FB7F8944091EA035091EB0360913B
:1028C000EC037091ED038FBF2FB7F8948091EA036A
:1028D0009091EB03A091EC03B091ED032FBF841B0B
:1028E000950BA60BB70B8E159F05A007B10760F3DC
:1028F0001F910F91FF90EF900895019759F0FC01FF
:10290000EE0FFF1FEE0FFF1F32978FB7F89431972E
:10291000F1F78FBF0895789484B5826084BD84B543
:10292000816084BD85B5826085BD85B5816085BDCA
:10293000EEE6F0E0808181608083E1E8F0E0808174
:1029400082608083808181608083E0E8F0E0808124
:1029500081608083E1EBF0E0808184608083E0EB44
:10296000F0E0808181608083EAE7F0E0808184602C
:102970008083808182608083808181608083808188
:10298000806880831092C10008958093210108958A
:102990008F70909121019295990F990F907C982BAF
:1029A00090937C0080917A00806480937A0080917B
:1029B0007A0086FDFCCF2091780040917900942F19
:1029C00080E030E0282B392BC90108951F93CF9365
:1029D000DF93182FEB0161E00E943A15E12FF0E040
:1029E000E15EFE4F8491833051F4809180008068D5
:1029F00080938000D0938900C093880037C08430D2
:102A000051F480918000806280938000D0938B008D
:102A1000C0938A002BC0813029F484B5806884BDBE
:102A2000C7BD24C0823029F484B5806284BDC8BD8E
:102A30001DC0863041F48091B00080688093B00062
:102A4000C093B30013C0873041F48091B00080621E
:102A50008093B000C093B40009C0C038D10514F40D
:102A600060E001C061E0812F0E945815DF91CF9195
:102A70001F910895282F30E0C901855F9E4FFC010A
:102A8000949129503F4FF9018491882381F0E82FD8
:102A9000F0E0E851FF4FE491F0E0662329F48081F3
:102AA00090958923808308958081892B8083089560
:102AB000482F50E0CA01815E9E4FFC012491CA015B
:102AC000855F9E4FFC01949149505F4FFA0134910C
:102AD0003323C1F1222331F1233021F4809180008E
:102AE0008F7705C0243031F4809180008F7D8093F2
:102AF000800018C0213019F484B58F7704C02230CB
:102B000021F484B58F7D84BD0DC0263021F48091E1
:102B1000B0008F7705C0273029F48091B0008F7DF9
:102B20008093B000E32FF0E0E351FF4FE491F0E039
:102B3000662329F48081909589238083089580817C
:102B4000892B80830895482F50E0CA01815E9E4FF3
:102B5000FC012491CA01855F9E4FFC01949149506C
:102B60005F4FFA013491332319F420E030E035C08F
:102B7000222331F1233021F4809180008F7705C02A
:102B8000243031F4809180008F7D8093800018C0C4
:102B9000213019F484B58F7704C0223021F484B534
:102BA0008F7D84BD0DC0263021F48091B0008F77D9
:102BB00005C0273029F48091B0008F7D8093B0004C
:102BC000E32FF0E0EE50FF4FE491F0E0808120E051
:102BD00030E0892311F021E030E0C9010895EF923F
:102BE000FF920F931F937B018C0122E030E040E0C5
:102BF00050E00E943417205C3D4B404F5F4FCA01AC
:102C0000B901A80197010E943417C901DA0101979F
:102C1000A109B109292F3A2F4B2F552747FD5A9566
:102C20000196A11DB11D2093C50081508093C40061
:102C3000E1ECF0E080818061808380818860808326
:102C40008081806880831F910F91FF90EF9008959D
:102C5000982F8091C00085FFFCCF9093C600089507
:102C60008091EE039091EF0380589F4F2091F003E5
:102C70003091F103821B930B60E870E00E94FF1615
:102C800008954091F0035091F1038091EE039091EB
:102C9000EF038417950719F42FEF3FEF0FC0FA01E8
:102CA000EE50FC4F2081CA01019660E870E00E945E
:102CB000FF169093F1038093F00330E0C90108956B
:102CC0008091F0039091F1039093EF038093EE03D2
:102CD00008951F920F920FB60F9211242F933F93D6
:102CE0004F935F936F937F938F939F93AF93BF9314
:102CF000EF93FF934091C600E091EE03F091EF0354
:102D0000CF01019660E870E00E94FF169C0180915F
:102D1000F0039091F1032817390739F0EE50FC4F7A
:102D200040833093EF032093EE03FF91EF91BF9127
:102D3000AF919F918F917F916F915F914F913F9153
:102D40002F910F900FBE0F901F901895FB01DC0183
:102D50008D91019080190110D9F3990B0895FB0111
:102D6000DC014150504030F08D910190801919F4F0
:102D70000020B9F7881B990B0895FB01DC01415035
:102D8000504048F001900D920020C9F701C01D92FB
:102D900041505040E0F70895629FD001739FF001C9
:102DA000829FE00DF11D649FE00DF11D929FF00DDB
:102DB000839FF00D749FF00D659FF00D9927729F12
:102DC000B00DE11DF91F639FB00DE11DF91FBD019D
:102DD000CF0111240895AA1BBB1B51E107C0AA1FF4
:102DE000BB1FA617B70710F0A61BB70B881F991FAC
:102DF0005A95A9F780959095BC01CD01089597FB50
:102E0000092E07260AD077FD04D0E5DF06D0002082
:102E10001AF4709561957F4F0895F6F79095819516
:102E20009F4F0895A1E21A2EAA1BBB1BFD010DC0E6
:102E3000AA1FBB1FEE1FFF1FA217B307E407F5076A
:102E400020F0A21BB30BE40BF50B661F771F881F46
:102E5000991F1A9469F760957095809590959B01DC
:102E6000AC01BD01CF01089597FB092E05260ED0B8
:102E700057FD04D0D7DF0AD0001C38F45095409598
:102E8000309521953F4F4F4F5F4F0895F6F790953E
:102E90008095709561957F4F8F4F9F4F0895EE0FEE
:0E2EA000FF1F0590F491E02D0994F894FFCFE8
:102EAE00FFFF52494646005741564500666D742055
:102EBE0000414C41524D2E57415600000000004734
:022ECE001201EF
:00000001FF
